:020000040000FA
:060000002CEF21F01200BC
:020006001200E6
:080008000000000000000000F0
:0700100000000000000000E9
:060018004CEF1AF012008B
:02001E000300DD
:1000200010000000080E000007000000080000009B
:10003000000E000008000000AC420000CF010000EC
:0400400015000000A7
:0C004400D9CFE6FFE1CFD9FF0B0EE1267B
:10005000DF6A010EDB6A040EF36E020EF3CFDBFFE4
:10006000010EF36E030EF3CFDBFF080EF36E040EEA
:10007000F3CFDBFF060EF36E050EF3CFDBFF010EB1
:10008000F36E060EF3CFDBFF010EF36E070EF3CF18
:10009000DBFF010EF36E080EF3CFDBFF090EDB6A08
:1000A0000A0EDB6AD398D38AD38C9B9CC26A300E2B
:1000B000C16E920EC06E0F010B0E5D6F5C6BC28045
:1000C000928092829286898A929AFB0E936E949085
:1000D000949294948C6A956A96909692030E8D12DF
:1000E000F80E8B148B6E8B802EEC0CF052EC0DF016
:1000F000010EF1C1DBFFD950010FE66E000EDA20D0
:10010000E66E89EC0DF0E552E552DF6ADFCF14F0C0
:10011000180EE76E1418E8AE02D0E73402D0E750AC
:10012000145C1BE2DFCFE9FFEA6AE9BEEA68D89017
:10013000E936EA36520EE926020EEA22EE68ED684A
:10014000DFCFE9FFEA6AE9BEEA68900EE926020E0F
:10015000EA22CD0EEF6EDF2AD9D7E668E668E668B8
:10016000E66AE66AE66AE66AE66A010EE66EE3ECCD
:1001700005F0146E090EE15E14500201BC6BF28EA4
:10018000F28C0B0EE15C02E2E16AE552E16EE552AF
:10019000E7CFD9FF1200D9CFE6FFE1CFD9FFE65272
:1001A000DF6AFD0EDBCFE9FFFE0EDBCFEAFFEECF0D
:1001B00008F0EDCF09F00850100B23E082A821D001
:1001C000100EE66EE66AB00EE66E100EE66EFEECFF
:1001D00008F0E552E552E552E552000902E002015D
:1001E000BC2BFD0EDBCFE9FFFE0EDBCFEAFFEE9866
:1001F000ED52FD0EDBCFE9FFFE0EDBCFEAFFEE8A0C
:10020000ED52FD0EDBCFE9FFFE0EDBCFEAFFEECFB6
:1002100008F0EDCF09F00850200B1BE082A819D0A0
:10022000200EE66EE66AB00EE66E100EE66EFEEC8E
:1002300008F0E552E552E552E552000902E00201FC
:10024000BC2BFD0EDBCFE9FFFE0EDBCFEAFFEE9A03
:10025000ED52FD0EDBCFE9FFFE0EDBCFEAFFEECF66
:1002600008F0EDCF09F00850400B23E082A821D020
:10027000400EE66EE66A500EE66E300EE66E20EC3C
:100280000AF0E552E552E552E552000902E00201AA
:10029000BC2BFD0EDBCFE9FFFE0EDBCFEAFFEE8EBF
:1002A000ED52FD0EDBCFE9FFFE0EDBCFEAFFEE9C49
:1002B000ED52FD0EDBCFE9FFFE0EDBCFEAFFEECF06
:1002C00008F0EDCF09F00850800B33E082A831D060
:1002D000800EE66EE66A500EE66E300EE66E20EC9C
:1002E0000AF0E552E552E552E552000902E002014A
:1002F000BC2B070E8B14DF6EF80E8B148B6EDFCFCA
:1003000014F0060EE76E1418E8AE02D0E73402D0FF
:10031000E750145C04E2DF508B10010F01D0010E96
:100320008B6EFD0EDBCFE9FFFE0EDBCFEAFFEE9E0C
:10033000ED6AE552E552E7CFD9FF1200D9CFE6FFCB
:10034000E1CFD9FF040EE126010EDE6EDE6ADE6A21
:10035000DD6ADD52DD52DECF14F0DECF15F0DECFE8
:1003600016F0DDCF17F0DD52DD52FE0EDB5008E057
:100370000001D8901436153616361736E804F9E120
:1003800014C0DFFF010E15C0DBFF020E16C0DBFF3D
:10039000030E17C0DBFFE66AE66AE66AE66AD9CFB3
:1003A000E9FFDACFEAFFEECFE6FFEECFE6FFEECFD2
:1003B000E6FFEFCFE6FF010EE66EE3EC05F0146E0C
:1003C000090EE15E1450040EE15C02E2E16AE552BE
:1003D000E16EE552E7CFD9FF1200D9CFE6FFE1CFBA
:1003E000D9FF040EE126010EDE6EDE6ADE6ADD6AEA
:1003F000DD52DD52DECF14F0DECF15F0DECF16F089
:10040000DDCF17F0DD52DD52FE0EDB5008E00001BB
:10041000D8901436153616361736E804F9E114C0AC
:10042000DFFF010E15C0DBFF020E16C0DBFF030E5F
:1004300017C0DBFFD9CFE9FFDACFEAFFEECFE6FF47
:10044000EECFE6FFEECFE6FFEFCFE6FFE66AE66A25
:10045000E66AE66A010EE66EB6DB146E090EE15E30
:100460001450040EE15C02E2E16AE552E16EE552ED
:10047000E7CFD9FF1200E6680F0EE66EE66AE66A7D
:10048000E66AE66AE66AE66AE66A9DDB146E090ECB
:10049000E15E14501200D9CFE6FFE1CFD9FF020E82
:1004A000E126FE0EEA6ADB34FE0BEA36E96E520EF6
:1004B000E926020EEA22EECFDEFFEDCFDDFF0E01D0
:1004C0000E5125E1DECF14F0DDCF15F0D890155098
:1004D00004E6030E145C000E155819E3DECF14F089
:1004E000DDCF15F0153411E21450F0080A0E155442
:1004F0000CE2DECF16F0DDCF17F0D890175004E6EF
:10050000100E165C0E0E175802E3010E0E6FFE0E53
:10051000EA6ADB34FE0BEA36E96E520EE926020E79
:10052000EA22EE68ED68DECF14F0DDCF15F014C0DE
:10053000F3FF15C0F4FF020EE15C02E2E16AE5524E
:10054000E16EE552E7CFD9FF1200D9CFE6FFE1CF48
:10055000D9FFE652FE0EDB50EA6A900FE96E020EFA
:10056000EA22EFCFDFFF0E010D5127E1DFCF14F0BC
:10057000D30EE76E1418E8AE02D0E73402D0E7508D
:10058000145C1BE3DFCF14F00A0EE76E1418E8AE1C
:1005900002D0143403D0E750D88014540CE2DFCFDB
:1005A00015F0320EE76E1518E8AE02D0E73402D02F
:1005B000E750155C02E3010E0D6FFE0EDB50EA6A98
:1005C000900FE96E020EEA22CD0EEF6EDFCF14F02F
:1005D000156A14BE156814C0F3FF15C0F4FFE55288
:1005E000E552E7CFD9FF1200D9CFE6FFE1CFD9FF1F
:1005F000FD0EDBCFE9FFFE0EDBCFEAFFEE6AED6A10
:10060000D80E0201E76EA819E8AE02D0E73402D096
:10061000E750A85D08E2FD0EDBCFE9FFFE0EDBCF61
:10062000EAFFEE80ED52D80EE76EA919E8AE02D0CF
:10063000E73402D0E750A95D08E2FD0EDBCFE9FF09
:10064000FE0EDBCFEAFFEE82ED52500EE76EA819E8
:10065000E8AE02D0A83503D0E750D880A85508E20C
:10066000FD0EDBCFE9FFFE0EDBCFEAFFEE84ED529D
:10067000500EE76EA919E8AE02D0A93503D0E750B5
:10068000D880A95508E2FD0EDBCFE9FFFE0EDBCFD7
:10069000EAFFEE86ED52AA5108E0FD0EDBCFE9FF3E
:1006A000FE0EDBCFEAFFEE88ED52AB5108E0FD0E07
:1006B000DBCFE9FFFE0EDBCFEAFFEE8AED520E0143
:1006C0000251031108E0FD0EDBCFE9FFFE0EDBCF88
:1006D000EAFFEE8CED52026B036B0201BC5108E0A5
:1006E000FD0EDBCFE9FFFE0EDBCFEAFFEE8EED5213
:1006F00080B408D0FD0EDBCFE9FFFE0EDBCFEAFFB2
:10070000EE52ED80FD0EDBCFE9FFFE0EDBCFEAFF00
:10071000020EE926000EEA22BCC2EFFFBC6BFD0E02
:10072000DBCFE9FFFE0EDBCFEAFF040EE926000E69
:10073000EA2200CEEEFF01CEEDFFE552E7CFD9FF72
:100740001200D9CFE6FFE1CFD9FF020EE126DE6A23
:10075000DD6A830EC2140C09C26EC282C2B2FED719
:10076000C450176E166AC35000011624146E000E92
:100770001720156E14C0DEFFDD6ED9CFE9FFDACF8A
:10078000EAFFF40EEE5E010EED5AD9CFE9FFDACFA3
:10079000EAFF0A0E0D6E0E6AEECF08F0EDCF09F0FB
:1007A00019EC1FF008C0EEFF09C0EDFFFD0EDBCF16
:1007B000E9FFFE0EDBCFEAFF030EE926000EEA2278
:1007C000DFCFEFFF020EE15C02E2E16AE552E16E8B
:1007D000E552E7CFD9FF1200D9CFE6FFE1CFD9FF2D
:1007E000E652DF6A0E01006B016B600EE66EDFEC15
:1007F00020F0E552100EE66EE66A9A0EE66E1E0EC8
:10080000E66EFEEC08F0E552E552E552E552600E68
:10081000E66EDFEC20F0E552200EE66EE66A9A0EF8
:10082000E66E1E0EE66EFEEC08F0E552E552E5526D
:10083000E552000903E00E01008F2BD0020EDF6E9F
:10084000DFCF14F0140EE76E1418E8AE02D0E734D0
:1008500002D0E750145C1DE2DFCFE9FFEA6AE9BE8F
:10086000EA682A0EE926020EEA22EF0402E10E01EE
:100870000081130EDF24E96EEA6AE9BEEA682A0EF7
:10088000E926020EEA22EF0402E10E010181DF2ACD
:10089000D7D7100EE66EE66A9D0EE66E1F0EE66E68
:1008A000FEEC08F0E552E552E552E552600EE66EC8
:1008B000DFEC20F0E552200EE66EE66A9D0EE66E55
:1008C0001F0EE66EFEEC08F0E552E552E552E552E9
:1008D000000903E00E01008F2BD0020EDF6EDFCF88
:1008E00014F0140EE76E1418E8AE02D0E73402D00C
:1008F000E750145C1DE2DFCFE9FFEA6AE9BEEA686F
:100900002A0EE926020EEA22EF0402E10E0100831C
:10091000130EDF24E96EEA6AE9BEEA682A0EE926C8
:10092000020EEA22EF0402E10E010183DF2AD7D78B
:10093000100EE66EE66AB00EE66E100EE66EFEEC87
:1009400008F0E552E552E552E552600EE66EDFEC46
:1009500020F0E552200EE66EE66AB00EE66E100E4E
:10096000E66EFEEC08F0E552E552E552E55200096C
:1009700002E00E01008F400EE66EE66A7A0EE66E29
:100980003E0EE66E20EC0AF0E552E552E552E552E5
:10099000140EE66EDFEC20F0E552800EE66EE66A9D
:1009A0007A0EE66E3E0EE66E20EC0AF0E552E55257
:1009B000E552E552000903E00E01008F35D0020E2A
:1009C000DF6EDFCF14F0060EE76E1418E8AE02D02B
:1009D000E73402D0E750145C1DE2DFCFE9FFEA6A9A
:1009E000E9BEEA68820EE926020EEA22EF0402E17D
:1009F0000E010085060EDF24E96EEA6AE9BEEA68A8
:100A0000820EE926020EEA22EF0402E10E010185C0
:100A1000DF2AD7D70201880502E10E010085020115
:100A20008E0502E10E010185400EE66EE66A7D0E3E
:100A3000E66E3F0EE66E20EC0AF0E552E552E55216
:100A4000E552140EE66EDFEC20F0E552800EE66E05
:100A5000E66A7D0EE66E3F0EE66E20EC0AF0E55289
:100A6000E552E552E552000903E00E01008F35D052
:100A7000020EDF6EDFCF14F0060EE76E1418E8AE3C
:100A800002D0E73402D0E750145C1DE2DFCFE9FF6B
:100A9000EA6AE9BEEA68820EE926020EEA22EF045B
:100AA00002E10E010087060EDF24E96EEA6AE9BE64
:100AB000EA68820EE926020EEA22EF0402E10E0144
:100AC0000187DF2AD7D70201880502E10E010087DE
:100AD00002018E0502E10E010187400EE66EE66A14
:100AE000500EE66E300EE66E20EC0AF0E552E5524E
:100AF000E552E552140EE66EDFEC20F0E552800E72
:100B0000E66EE66A500EE66E300EE66E20EC0AF0F7
:100B1000E552E552E552E552000902E00E01008F70
:100B2000100EE66EE66AD6DAE552E5526E0EE66E15
:100B3000DFEC20F0E552200EE66EE66ACBDAE552F5
:100B4000E552000903E00E01008F34D00201D89075
:100B5000B55104E6340EB45D080EB55902E20E013B
:100B600000890201B53507E2B45154080B0EB555A2
:100B700002E20E01008B0201B85102E00E01008D6D
:100B80000201D890B75104E6340EB65D080EB7598D
:100B900002E20E0101890201B73507E2B65154089D
:100BA0000B0EB75502E20E01018B0201B95102E0B2
:100BB0000E01018D00CEF3FF01CEF4FFE552E552A8
:100BC000E7CFD9FF1200D9CFE6FFE1CFD9FF180E4A
:100BD000E126140EDB6A150EDB6A160EDB6A170EB1
:100BE000DB6AD950FA0FE96EFF0EDA20EA6E0E01C9
:100BF0000451EE10046F0551EE10056F0651EE1012
:100C0000066F0751EE10076FF60EDBCF14F0F70EEC
:100C1000DBCF15F0F80EDBCF16F0F90EDBCF17F0B7
:100C2000141E151E161E171E040EE96E0E0EEA6E19
:100C3000EE501414046FEE501514056FEE50161498
:100C4000066FEE501714076F140E04CEDBFF150E5F
:100C500005CEDBFF160E06CEDBFF170E07CEDBFF41
:100C6000140EDBCF14F0150EDBCF15F0160EDBCF14
:100C700016F0170EDBCF17F01450E76E020EE7CF19
:100C8000DBFF140EDBCF14F0150EDBCF15F0160EC4
:100C9000DBCF16F0170EDBCF17F0080ED890173207
:100CA000163215321432E806F9E1140E14C0DBFFD7
:100CB000150E15C0DBFF160E16C0DBFF170E17C092
:100CC000DBFF0F0E146E156A166A176AD950140FDF
:100CD000E96EDACFEAFFEE501416EE501516EE501C
:100CE0001616EE501716030E14C0DBFF140EDBCFE2
:100CF00014F0150EDBCF15F0160EDBCF16F0170E25
:100D0000DBCF17F0040ED89017321632153214329A
:100D1000E806F9E1140E14C0DBFF150E15C0DBFF69
:100D2000160E16C0DBFF170E17C0DBFF140EDBCF4D
:100D300014F0150EDBCF15F0160EDBCF16F0170EE4
:100D4000DBCF17F01450DF6E140EDBCF14F0150E4E
:100D5000DBCF15F0160EDBCF16F0170EDBCF17F03A
:100D6000080ED8901732163215321432E806F9E11F
:100D7000140E14C0DBFF150E15C0DBFF160E16C0D7
:100D8000DBFF170E17C0DBFF0F0E146E156A166A15
:100D9000176AD950140FE96EDACFEAFFEE50141635
:100DA000EE501516EE501616EE501716010E14C022
:100DB000DBFFFE0EDB50100FE76E060EE7CFDBFF0A
:100DC000070EDFCFDBFF010EDB50E76E080EE7CF2B
:100DD000DBFF090EDB6A770EF36E0A0EF3CFDBFF43
:100DE000AA0EF36E0B0EF3CFDBFF060EE66ED950A4
:100DF000060FE66E000EDA20E66E7AEC0BF0E55296
:100E0000E552E552E76E0C0EE7CFDBFFFE0EDB503E
:100E1000100FE76E0D0EE7CFDBFF020EDB50E76E23
:100E20000E0EE7CFDBFF030EDB50E76E0F0EE7CFB2
:100E3000DBFF100EDB6A770EF36E110EF3CFDBFFD4
:100E4000AA0EF36E120EF3CFDBFF060EE66ED9503C
:100E50000D0FE66E000EDA20E66E7AEC0BF0E5522E
:100E6000E552E552E76E130EE7CFDBFFD950040FD2
:100E7000E66E000EDA20E66E100EE66EC70EE66E27
:100E8000010EE66E08EC0DF0146E050EE15E1450D6
:100E9000180EE15C02E2E16AE552E16EE552E7CF4D
:100EA000D9FF1200D9CFE6FFE1CFD9FFE652DF6AC2
:100EB000000EE66E020EE66E100EE66ECE0EE66ECA
:100EC000020EE66E08EC0DF0146E050EE15E145095
:100ED000060EE66E020EE66E020EE66E7AEC0BF081
:100EE000E552E552E5520201085D0EE1060EE66E9E
:100EF000090EE66E020EE66E7AEC0BF0E552E55254
:100F0000E55202010F5D02E0DF6ADED0070E09152F
:100F1000116F070E0215106F0951E840E840E840D4
:100F20001F0B010B136F0251E840E840E8401F0B14
:100F3000010B126F09390F0B010B156F02390F0BE3
:100F4000010B146F0951E00BE838E840030B176FF1
:100F50000251E00BE838E840030B166F0945010B1E
:100F6000010B196F0245010B010B186F0F0E0B15CA
:100F70001C6F1D6B156E146A0A5114241C6F000E31
:100F800015201D6F0F0E04151A6F1B6B156E146A5A
:100F9000035114241A6F000E15201B6F0C51206F83
:100FA000216B0CC214F021C215F0040ED890143637
:100FB0001536E804FBE102010B390F0B1424206FF6
:100FC000000E1520216F05511E6F1F6B05C214F016
:100FD0001FC215F0040ED89014361536E804FBE154
:100FE000020104390F0B14241E6F000E15201F6F11
:100FF0001F0E0D5D246F256B040E000A06E0020132
:10100000D89024372537E804FBE124C214F025C228
:1010100015F0D89015321432020124511424246F93
:1010200025511520256F1F0E065D226F236B040EC0
:10103000000A06E00201D89022372337E804FBE1DA
:1010400022C214F023C215F0D890153214320201D6
:1010500022511424226F23511520236F200E0E5D80
:10106000286F296B040E000A06E00201D890283789
:101070002937E804FBE128C214F029C215F0D89002
:1010800015321432020128511424286F29511520D9
:10109000296F200E075D266F276B040E000A06E0FD
:1010A0000201D89026372737E804FBE126C214F066
:1010B00027C215F0D890153214320201265114249B
:1010C000266F27511520276FDF50E552E552E7CFF5
:1010D000D9FF1200D9CFE6FFE1CFD9FFE652DF6A90
:1010E000D950FD0FE96EFF0EDA20EA6E100EEE18F1
:1010F0000AE1ED5008E1790EE66E520EE66EF3EC71
:101100000CF0E552E552D950FD0FE96EFF0EDA20E2
:10111000EA6E200EEE186CE1ED506AE182A868D00C
:10112000898AAC0EE66E020EE66E080EE66E6B0E57
:10113000E66E540EE66E08EC0DF0146E050EE15EE0
:101140001450020EE66EAE0EE66E020EE66ED2DAB7
:10115000E552E552E5520201B05D0DE1020EE66E88
:10116000B10EE66E020EE66EC5DAE552E552E552C4
:101170000201B35D02E0DF6A3BD0AFC2E6FFAEC260
:10118000E6FF73DBE552E552F3CFB4F2F4CFB5F2EC
:10119000B2C2E6FFB1C2E6FF68DBE552E552F3CF2B
:1011A000B6F2F4CFB7F20201AF51E00BE838E840F5
:1011B000010BB86FB251E00BE838E840010BB96F92
:1011C000060EAFC2E7FF070B04E0E742E79EE80622
:1011D000FCE1E7500201BA6F060EB2C2E7FF070B4F
:1011E00004E0E742E79EE806FCE1E7500201BB6F3E
:1011F000DF50E552E552E7CFD9FF1200D9CFE6FF25
:10120000E1CFD9FF030EE126020EDB6AD950FB0FB6
:10121000E96EFF0EDA20EA6E100EEE181AE1ED50BC
:1012200018E1E668E668E668E66AE66AE66AE66A9B
:10123000E66A010EE66EC7DC146E090EE15E14501C
:10124000FD0EDBCFE6FFFE0EDBCFE6FFCCDBE5528B
:10125000E552D950FB0FE96EFF0EDA20EA6E200E40
:10126000EE1801E0DFD0ED5001E0DCD082A8DAD04A
:10127000898ACFC114F0D0C115F0D1C116F0D2C106
:1012800017F0141E151E161E171E14C0E6FF15C0FB
:10129000E6FF16C0E6FF17C0E6FFCFC1E6FFD0C1EC
:1012A000E6FFD1C1E6FFD2C1E6FF010EE66E8BDCA0
:1012B000186E090EE15E18502A0EE66E020EE66EFA
:1012C000280EE66EDC0EE66E040EE66EA1DB146EF2
:1012D000050EE15E1450120EE66E2C0EE66E020E46
:1012E000E66E08DAE552E552E55202013E5D0DE197
:1012F000120EE66E3F0EE66E020EE66EFBD9E5526A
:10130000E552E5520201515D03E0020EDB6A8AD02C
:10131000DF6ADFCF14F0180EE76E1418E8AE02D0C3
:10132000E73402D0E750145C01E37CD0DF407F0B50
:10133000DF24E76E010EE7CFDBFFDFCF14F00B0EEB
:10134000E76E1418E8AE02D0143403D0E750D8800A
:10135000145402E2010EDB2A010EDB50030FE96E8A
:10136000EA6AE9BEEA682A0EE926020EEA22EF508E
:10137000E66E010EDB50020FE96EEA6AE9BEEA682A
:101380002A0EE926020EEA22EF50E66E6EDAE552E8
:10139000E552F3CF14F0F4CF15F0DFCFE9FFEA6A9E
:1013A000E9BEEA68D890E936EA36520EE926020E1E
:1013B000EA2214C0EEFF15C0EDFF010EDB50040F52
:1013C000E96EEA6AE9BEEA682A0EE926020EEA2216
:1013D000EF50E66E010EDB50030FE96EEA6AE9BEDC
:1013E000EA682A0EE926020EEA22EF50E66E9BDA40
:1013F000E552E552F3CF14F0F4CF15F0DF28E96E93
:10140000EA6AE9BEEA68D890E936EA36520EE92679
:10141000020EEA2214C0EEFF15C0EDFF020EDF241B
:10142000DF6E77D7020EDB50146E030EE15C02E232
:10143000E16AE552E16E1450E552E7CFD9FF1200A0
:10144000D9CFE6FFE1CFD9FF070EE126040EDB6A14
:10145000050EDB6A060EDB6AD950FB0FE96EFF0E44
:10146000DA20EA6E400EEE180BE1ED5009E1FD0EB8
:10147000DBCFE6FFFE0EDBCFE6FFB5DAE552E55245
:10148000D950FB0FE96EFF0EDA20EA6E800EEE18DF
:1014900001E022D1ED5001E01FD182A81DD1898A3F
:1014A000820EE66E020EE66E0E0EE66EEA0EE66E38
:1014B0000E0EE66EADDA146E050EE15E1450050EEA
:1014C000E66E840EE66E020EE66E14D9E552E55223
:1014D000E5520201895D0DE1050EE66E8A0EE66EAB
:1014E000020EE66E07D9E552E552E55202018F5D24
:1014F00003E0060EDB6AF0D0DE52020EDD6E070E50
:101500008B14E76E040EE7CFDBFFDB06DBCFE6FFD5
:10151000050EE552D880E754E76E050EE7CFDBFFF6
:10152000DF6ADFCF14F0180EE76E1418E8AE02D0B1
:10153000E73402D0E750145C01E3C5D0010EDB288C
:10154000E96EEA6AE9BEEA68820EE926020EEA223C
:10155000EF50E66E010EDBCFE9FFEA6AE9BEEA680A
:10156000820EE926020EEA22EF50E66E7ED9E5529F
:10157000E552020EF3CFDBFF030EF4CFDBFF020ECA
:10158000DBCFE6FF030EDBCFE6FF6EEC20F0E5528B
:10159000E552E66E040EDB50E824DF24EA6A900F81
:1015A000E96E020EEA22E552E750EF6E010EDB2AE9
:1015B000DB28E96EEA6AE9BEEA68820EE926020ED5
:1015C000EA22EF50E66E010EDBCFE9FFEA6AE9BEE0
:1015D000EA68820EE926020EEA22EF50E66EA3D9EF
:1015E000E552E552020EF3CFDBFF030EF4CFDBFF33
:1015F000020EDBCFE6FF030EDBCFE6FF6EEC20F042
:10160000E552E552E66E050EDB50E824DF24010FBB
:10161000EA6A900FE96E020EEA22E552E750EF6E99
:10162000010EDB50020FE76E010EE7CFDBFFDB2878
:10163000E96EEA6AE9BEEA68820EE926020EEA224B
:10164000EF50E66E010EDBCFE9FFEA6AE9BEEA6819
:10165000820EE926020EEA22EF50E66E06D9E55226
:10166000E552020EF3CFDBFF030EF4CFDBFF020ED9
:10167000DBCF15F0030EDBCF16F0D8901632153203
:10168000E804FBE1110E155E010E165A0C0E146EE5
:101690000E6EDFCF09F0FFEC1EF009C0E9FFEA6A29
:1016A000E9BEEA68A80EE926020EEA2215C0EFFF9D
:1016B000010EDB50030FE76E010EE7CFDBFF0C0ED0
:1016C000DF24DF6E2ED7020188390F0B010BAA6FC2
:1016D0008E390F0B010BAB6F060EDB50146E070E2D
:1016E000E15C02E2E16AE552E16E1450E552E7CFB7
:1016F000D9FF1200D9CFE6FFE1CFD9FF070EE126CF
:10170000410EF36E020EF3CFDBFF030EDB6A040E15
:10171000DB6A050EDB6A060EDB6ADF6AFC0EDB5055
:10172000DF5C01E38DD0010EDB6ADBCF14F0080E25
:10173000E76E1418E8AE02D0E73402D0E750145C2C
:1017400001E37CD0800E156E010EDB5015C0E7FF63
:10175000070B04E0E742E79EE806FCE1E750146E61
:10176000DF50E76EFD0EDBCFE9FFFE0EDBCFEAFFB9
:10177000E750E926000EEA22EF501414E76E030E3C
:10178000E7CFDBFF010EDBCFE6FF070EE552D88087
:10179000E754146E030EDB5014C0E7FFE75204E079
:1017A000E8427F0BE706FCE1E76E030EE7CFDBFFC5
:1017B000DBCFE6FF020EDB50800BE844010BE55265
:1017C000E718E76E040EE7CFDBFFDBCFE6FF020E84
:1017D000DB50010BE552E718E76E050EE7CFDBFFA4
:1017E000040EDBCFE6FF020EDB50020BE8407F0B5E
:1017F000E552E718E76E060EE7CFDBFF020EDB507F
:10180000020D020EF3CFDBFF040EDBCFE6FF050E69
:10181000DB50E824156E060EDB50040DF350151056
:10182000E552E710146E020EDB50F80B1410E76E51
:10183000020EE7CFDBFF010EDB2A77D7DF2A6ED758
:10184000020EDB50146E070EE15C02E2E16AE55223
:10185000E16E1450E552E7CFD9FF12009496949AA6
:10186000320EC66EC79C9E961200D9CFE6FFE1CF1E
:10187000D9FF020EE126DE6ADD6AFD0EDB500F0B9A
:10188000DE6EDD6ADECF16F0DDCF17F016C017F082
:10189000166AFE0EDB501624146E000E172014C0BC
:1018A000DEFFDD6EDECF14F0DDCF15F0000E145E2E
:1018B000020E155A14C0DEFF15C0DDFFDECF14F096
:1018C000DDCF15F0800E151408E1DECF16F0DDCF68
:1018D00017F0D890173216320BD0DECF16F0DDCFCE
:1018E00017F0D89017321632000E1626800E1722E7
:1018F000DE501624146EDD501720156E14C0DEFF66
:10190000DD6EDECF14F0DDCF15F014C0F3FF15C08F
:10191000F4FF020EE15C02E2E16AE552E16EE5529B
:10192000E7CFD9FF1200D9CFE6FFE1CFD9FF020EF2
:10193000E126DE6ADD6AFD0EDB50DE6EDD6ADECF9B
:1019400016F0DDCF17F0040ED89016361736E804DF
:10195000FBE1FE0EDB380F0B1624146E000E172071
:1019600014C0DEFFDD6EDECF14F0DDCF15F0000E0B
:10197000145E020E155A14C0DEFF15C0DDFFDECF67
:1019800014F0DDCF15F0800E151408E1DECF16F04F
:10199000DDCF17F0D890173216320BD0DECF16F00D
:1019A000DDCF17F0D89017321632000E1626800EB3
:1019B0001722DE501624146EDD50172014C0DEFFEF
:1019C000DD6EDECF14F0DDCF15F014C0F3FF15C0CF
:1019D000F4FF020EE15C02E2E16AE552E16EE552DB
:1019E000E7CFD9FF1200D9CFE6FFE1CFD9FF899A1F
:1019F000FE0EDB50C96E9EA6FED79E96FD0EDB50F6
:101A0000C96E9EA6FED79E96E552E7CFD9FF12007B
:101A1000D9CFE6FFE1CFD9FFE652FA0EDBCFE9FFDF
:101A2000FB0EDBCFEAFFFE0EDBCFEFFF010EE76E12
:101A3000FA0EDBCFE9FFFB0EDBCFEAFFE750E9262A
:101A4000000EEA22FD0EDBCFEFFF899ADF6AFC0E63
:101A5000DB50DF5C21E2DF50E76EFA0EDBCFE9FFFF
:101A6000FB0EDBCFEAFFE750E926000EEA22EF503B
:101A7000C96E9EA6FED79E96DF50E76EFA0EDBCFAC
:101A8000E9FFFB0EDBCFEAFFE750E926000EEA2272
:101A9000C9CFEFFFDF2ADBD7898AE552E552E7CFCE
:101AA000D9FF1200CD88CD8A9F909D809E90CD82D7
:101AB000CD8012000E01028D1200D9CFE6FFE1CFDA
:101AC000D9FF020EE126DE6ADD6A830EC214000928
:101AD000C26EC282C2B2FED7C450176E166AC3501D
:101AE0001624146E000E172014C0DEFFDD6EDECF4C
:101AF00014F0DDCF15F014C0F3FF15C0F4FF020E93
:101B0000E15C02E2E16AE552E16EE552E7CFD9FF1E
:021B10001200C1
:0E1B1200D9CFE6FFE1CFD9FF800EE66E75EC6D
:101B200018F0E552729E728CFD0EDBCFE9FFFE0EBF
:101B3000DBCFEAFFEE52EF04146EFD0EDBCFE9FFC0
:101B4000FE0EDBCFEAFF050EE926000EEA22EF04C7
:101B5000400DF35014100E01436FFD0EDBCFE9FF73
:101B6000FE0EDBCFEAFF020EE926000EEA22EF04AA
:101B7000166EFD0EDBCFE9FFFE0EDBCFEAFF030E94
:101B8000E926000EEA22EF04080DF3CF15F0FD0E52
:101B9000DBCFE9FFFE0EDBCFEAFF070EE926000EE2
:101BA000EA22EF50400DF3CF14F0FD0EDBCFE9FF3A
:101BB000FE0EDBCFEAFF060EE926000EEA22EF500A
:101BC000800DF350141015101610446FFD0EDBCF6E
:101BD000E9FFFE0EDBCFEAFF040EE926000EEA2243
:101BE000EF04156EFD0EDBCFE9FFFE0EDBCFEAFF43
:101BF000090EE926000EEA22EF50400DF3CF14F053
:101C0000FD0EDBCFE9FFFE0EDBCFEAFF080EE92673
:101C1000000EEA22EF50800DF35014101510456F9E
:101C20007D95E66AE668070EE66EE66AE66AF80EF5
:101C3000E66E0E0EE66E89EC18F0146E070EE15E8D
:101C400014500E01466B476B4681E66AFD0EDBCFF2
:101C5000E9FFFE0EDBCFEAFFEF50156A000F146EAE
:101C6000010E1522166A176A15AE02D0166817689B
:101C700014C0E6FF15C0E6FF16C0E6FF17C0E6FF7A
:101C8000E00EE66E0E0EE66E89EC18F0186E070E8A
:101C9000E15E18500E01FC0E796FF00E716F7269E3
:101CA000200E706EE66A75EC18F0E552606A0F015E
:101CB000306B0E01806BFD0EDBCFE9FFFE0EDBCF3C
:101CC000EAFFEF50E66EC5EC14F0E552010EE55266
:101CD000E7CFD9FF1200D9CFE6FFE1CFD9FFE65217
:101CE000FD0EDBCFE9FFFE0EDBCFEAFFEFCFDFFF1C
:101CF000DF50120DF3CFE9FFF4CFEAFF000EE92623
:101D0000010EEA22DFCFEFFFFD0EDBCFE9FFFE0E73
:101D1000DBCFEAFFEE52EECF14F0EECF15F0EECFB0
:101D200016F0EFCF17F0DF50120DF3CFE9FFF4CF2D
:101D3000EAFF000EE926010EEA22EE5214C0EEFF81
:101D400015C0EEFF16C0EEFF17C0EEFFFD0EDBCF95
:101D5000E9FFFE0EDBCFEAFF050EE926000EEA22C0
:101D6000EF50E66EDF50120DF3CFE9FFF4CFEAFF3C
:101D7000000EE926010EEA22050EE926000EEA22EF
:101D8000E552E750EF6EFD0EDBCFE9FFFE0EDBCF35
:101D9000EAFF060EE926000EEA22EECF14F0EECF9F
:101DA00015F0EECF16F0EFCF17F0DF50120DF3CF96
:101DB000E9FFF4CFEAFF000EE926010EEA22060E43
:101DC000E926000EEA2214C0EEFF15C0EEFF16C091
:101DD000EEFF17C0EEFF010EE552E552E7CFD9FF47
:101DE0001200D9CFE6FFE1CFD9FF020EE126DF6A6C
:101DF000010EDB6ADB6A320EF36E010EDBCFF4FFFD
:101E0000F350F45C33E2E66AFD0EDBCFE9FFFE0E31
:101E1000DBCFEAFF050EE926000EEA22EF50E66E60
:101E2000FB0EDBCFE6FFFC0EDBCFE6FFFD0EDBCFCC
:101E3000E9FFFE0EDBCFEAFFEE52EECFE6FFEECF7C
:101E4000E6FFEECFE6FFEFCFE6FFF2EC15F0146E03
:101E5000080EE15E1450DF6EDF5008E10B0EE66EF7
:101E60003AEC21F0E552010EDB2AC5D7DF50146EA3
:101E7000020EE15C02E2E16AE552E16E1450E552C5
:101E8000E7CFD9FF1200D9CFE6FFE1CFD9FF020E8D
:101E9000E126010EDB6AD9CFE6FFDACFE6FFFD0EC1
:101EA000DBCFE9FFFE0EDBCFEAFF050EE926000ED1
:101EB000EA22E9CF14F0EACF15F0E9CFE6FFEACF46
:101EC000E6FFFB0EDBCFE6FFFC0EDBCFE6FFFD0EF1
:101ED000DBCFE9FFFE0EDBCFEAFFEE52E9CF16F0D3
:101EE000EACF17F0E9CFE6FFEACFE6FF45EC17F0BF
:101EF000186E080EE15E1850E76E010EE7CFDBFFAB
:101F0000080EDF140101CE6F010EDB50146E020EBD
:101F1000E15C02E2E16AE552E16E1450E552E7CF7E
:101F2000D9FF1200D9CFE6FFE1CFD9FF040EE12699
:101F3000DF6A010EDB6A020EDB6A030EDB6ADF6A10
:101F4000DFCF14F0060EE76E1418E8AE02D0E734C7
:101F500002D0E750145C01E3B5D0040EDF02F35069
:101F6000E66E4BEC02F0E552020EF3CFDBFF030E00
:101F7000F4CFDBFF0101D551200DF350E00B01013F
:101F8000C66F020E030EDBCF17F017C016F0176AEC
:101F9000C65100011610E8CFC6F1FF0EE76E020E23
:101FA000DBCF14F0030EE7501416156A14C0C7F106
:101FB000040EDF02F328E66E4BEC02F0E552020E4F
:101FC000F3CFDBFF030EF4CFDBFF020E030EDBCFFC
:101FD00015F015C014F0156A14C0C8F1FF0EE76EB5
:101FE000020EDBCF14F0030EE7501416156A14C06E
:101FF000C9F1040EDF02F350020FE66E4BEC02F063
:10200000E552020EF3CFDBFF030EF4CFDBFF020E2F
:10201000030EDBCF15F015C014F0156A14C0CAF119
:10202000FF0EE76E020EDBCF14F0030EE75014161E
:10203000156A14C0CBF1040EDF02F350030FE66EF5
:102040004BEC02F0E552020EF3CFDBFF030EF4CFB0
:10205000DBFF020E030EDBCF15F015C014F0156A7E
:1020600014C0CCF1FF0EE76E020EDBCF14F0030EAE
:10207000E7501416156A14C0CDF1C60EE66E010EB7
:10208000E66EDF28146E156A14BE1568120E15026E
:10209000F3CF15F01402F3CF14F0F4501526000E10
:1020A0001426010E152214C0E6FF15C0E6FF99DEC6
:1020B000E552E552E552E552E76E010EE7CFDBFF50
:1020C000DF2A3ED7010EDB50146E040EE15C02E203
:1020D000E16AE552E16E1450E552E7CFD9FF1200F4
:1020E000D9CFE6FFE1CFD9FF080EE126060EDB6A65
:1020F000D9CFE6FFDACFE6FFA1EC03F0E552E552D7
:10210000030EDB50E76E070EE7CFDBFFDBCF14F0EB
:10211000000EE76E1418E8AE02D0143403D0E75076
:10212000D88014540DE2070EDBCF15F0460EE76E93
:102130001518E8AE02D0E73402D0E750155C03E38F
:102140000E01010E0C6F0101D651040DF3CF14F0F6
:102150000101D551200DF35014240101C66F070E63
:10216000DBCFC7F1040E0101D603F350E66EA5ECF8
:1021700002F0E552F3CFC8F1040E0101D603F328B3
:10218000E66EA5EC02F0E552F3CFC9F1040E0101B1
:10219000D603F350020FE66EA5EC02F0E552F3CF42
:1021A000CAF1040E0101D603F350030FE66EA5EC4D
:1021B00002F0E552F3CFCBF10101CC6BCD6BC60E33
:1021C000E66E010EE66E900EE66E010EE66E09DE1C
:1021D000E552E552E552E552E76E060EE7CFDBFF2A
:1021E000DB50146E080EE15C02E2E16AE552E16E3A
:1021F0001450E552E7CFD9FF1200D9CFE6FFE1CF67
:10220000D9FF090EE126080EDB6AD9CFE6FFDACF47
:10221000E6FF000EE66E010EE66E35DEE552E55293
:10222000E552E552000919E0010EF36E080EF3CFF6
:10223000DBFF8D70E00EDF14E00BE838E8400101B1
:10224000D86F1F0EDF140101D76FD8C1DAF1010179
:10225000DA2B080EDA5D01E3DA6B080EDB50146E40
:10226000090EE15C02E2E16AE552E16E1450E552CA
:10227000E7CFD9FF1200D9CFE6FFE1CFD9FF090E92
:10228000E126080EDB6AD9CFE6FFDACFE6FF000EC3
:10229000E66E010EE66EF7DDE552E552E552E552D7
:1022A000000976E0010EF36E080EF3CFDBFF7792A4
:1022B0008D70E00EDF14E00BE838E8400101D86FC4
:1022C0001F0EDF140101D76F0101DA510101D85D42
:1022D00003E10101DA2B06D0D8C1DAF10101DA2BD2
:1022E0000101DB2B080E0101DA5D01E3DA6B030E5D
:1022F000DBCFCFF10101D06BD16BD26B080E1F0B7E
:10230000CFC114F0D0C115F0D1C116F0D2C117F071
:1023100007E0D8901436153616361736E806F9E178
:10232000020EDBCF18F0196A1A6A1B6A14501824BF
:102330000101CF6F15501920D06F16501A20D16FA0
:1023400017501B20D26F080E1F0BCFC114F0D0C145
:1023500015F0D1C116F0D2C117F007E0D8901436AD
:10236000153616361736E806F9E1010EDBCF18F000
:10237000196A1A6A1B6A145018240101CF6F15508C
:102380001920D06F16501A20D16F17501B20D26F12
:10239000080EDB50146E090EE15C02E2E16AE552C0
:1023A000E16E1450E552E7CFD9FF1200D9CFE6FF16
:1023B000E1CFD9FF1C0EE126030EF36E080EF3CF1A
:1023C000DBFF090EDB6A0E0EF36E0A0EF3CFDBFFA6
:1023D0000B0EDB6A0C0EDB6A080EF36E0D0EF3CFEC
:1023E000DBFF0E0EDB6A0F0EDB6A100EDB6A110ECE
:1023F000DB6AD950120FE66E000EDA20E66ED95075
:102400000D0FE66E000EDA20E66ED9CFE6FFDACFCA
:10241000E6FFD9500E0FE66E000EDA20E66E45ECB0
:1024200017F0146E080EE15E1450E76E0C0EE7CF45
:10243000DBFF120EDB50080B0101CE6FD9500E0FDF
:10244000E96EDACFEAFFEE5065E1030EEE1862E1C5
:10245000EE5060E1EE505EE1070EDBCFE6FF060EC8
:10246000DBCFE6FF050EDBCFE6FF040EDBCFE6FF9A
:10247000030EDBCFE6FF020EDBCFE6FF010EDB50E3
:10248000DF18E552E718E552E718E552E718E5527C
:10249000E718E552E718E552E718E76E0B0EE7CFAD
:1024A000DBFF080EDB50F36E0B0EDB50F35C0CE130
:1024B0000101400EDD6F0101F16BF1C1E6FF65DA4C
:1024C000E552E66AF50E0CD0090EDB50F36E0B0EEA
:1024D000DB50F35C15E10101800EDD6FE66AF60E5C
:1024E000E66E0D0EE66EE66AE66AF80EE66E0E0E13
:1024F000E66E89EC18F0146E070EE15E14500AD0F7
:102500000A0EDB50F36E0B0EDB50F35C03E10101AE
:102510000A0EDD6F0101DD510A0A01E111D18A0ABB
:1025200001E183D0C00A01E012D1D9500E0FE96E4B
:10253000DACFEAFF0A0EEE1808E1010EEE1805E107
:10254000EE5003E1EE5001E110D9D9500E0FE96EC3
:10255000DACFEAFF0A0EEE1801E0F9D0030EEE180A
:1025600001E0F5D0EE5001E0F2D0EE5001E0EFD006
:10257000130EDB6A0D0EDB50F36E130EDBCFF4FF90
:10258000F350F45C20E2D9CF16F0DACF17F0130E37
:10259000DB500F01D924E96E000EDA20EA6EEF500D
:1025A000E66ED950140F146EDACF15F0130EDB500F
:1025B0001424E96E000EDA20EA6EE552E750EF6E61
:1025C000130EDB2AD7D7140EDB500101F25D01E0B8
:1025D000BED0150EDB50F35D01E0B9D0160EDB5016
:1025E000E95D01E0B4D0180EDB50EC5D01E0AFD046
:1025F0001B0EDBCFE6FFC9D9E552E66AE6680D0E91
:10260000E66EE66AE66AF80EE66E0E0EE66E89EC97
:1026100018F0146E070EE15E14501B0EDBCFE6FFC0
:102620000D0EE66EDEEC1EF088D0D9500E0FE96E6E
:10263000DACFEAFF090EEE1806E1030EEE1803E109
:10264000EE5001E1EE5002E0000E01D0010E146EDA
:10265000D9500E0FE96EDACFEAFF080EEE1806E148
:10266000030EEE1803E1EE5001E1EE5002E0000E21
:1026700001D0010E14106BE0130EDB6A0D0EDB505F
:10268000F36E130EDBCFF4FFF350F45C20E2D9CFEE
:1026900016F0DACF17F0130EDB500F01D924E96ED4
:1026A000000EDA20EA6EEF50E66ED950140F146E69
:1026B000DACF15F0130EDB501424E96E000EDA2089
:1026C000EA6EE552E750EF6E130EDB2AD7D7D950EA
:1026D0000E0FE96EDACFEAFF080EEE1814E1030ED2
:1026E000EE1811E1EE500FE1EE500DE1D950140F4C
:1026F000E66E000EDA20E66EE66A82EC1DF0E55228
:10270000E552E55224D0D9500E0FE96EDACFEAFF38
:10271000090EEE181CE1030EEE1819E1EE5017E158
:10272000EE5015E1D950140FE66E000EDA20E66E79
:10273000080EE66E82EC1DF0E552E552E55201D03E
:1027400014D80101200ED76F0101010EDD6F0C0EB0
:10275000DB50146E1C0EE15C02E2E16AE552E16EB0
:102760001450E552E7CFD9FF1200D9CFE6FFE1CFF1
:10277000D9FF060EE126DF6A010EDB6A020EDB6A74
:10278000030EDB6A040EDB6AF36E050EF3CFDBFF8C
:10279000F2C1C6F1F3C1C7F1E9C1C8F1F4C1C9F191
:1027A000ECC1CAF1F5C1CBF1EFC1CCF1F0C1CDF173
:1027B0000101F351E66ED950010FE96EDACFEAFF5D
:1027C000E552E750EE6EED6A010EDBCF14F0020E1B
:1027D00014C015F0146A010E14C0DBFF020E15C000
:1027E000DBFFF251E76E010EDBCF14F0020EDBCF00
:1027F00015F0E7501412010E14C0DBFF020E15C0D5
:10280000DBFF010EDB2A020E01E3DB2A030EDBCF26
:1028100014F0040EDBCF15F0010EDBCF16F0020E24
:10282000DBCF17F01450165C155017580CE3050E4B
:10283000DBCFE6FF0CEC21F0E552030EDB2A040EA1
:10284000E5E3DB2AE3D7C60EE66E010EE66EA20EC6
:10285000E66E010EE66EF1EC0EF0E552E552E55241
:10286000E552DF6EDF50146E060EE15C02E2E16AB3
:10287000E552E16E1450E552E7CFD9FF1200D9CFEF
:10288000E6FFE1CFD9FF070EE126060EDB6A0E0157
:10289000096B0A6B0B6BD9CFE6FFDACFE6FFF4ECDE
:1028A00002F0E552E552DECF14F0DDCF15F0400E18
:1028B0001416000E1516060ED89015321432E804C0
:1028C000FBE114C00AFE040EDBCF14F0050EDBCFD3
:1028D00015F0010E145C000E155803E30E01010EF5
:1028E0000B6F0101C66B0101D551200DF3500101A1
:1028F000D7250101C66FC76B0E010851400DF3CFFC
:10290000C7F10951200DF3500101C7130E010A3917
:10291000F00B0101C7130E010B51080DF35001011B
:10292000C7130E010C51040DF3500101C7130E0122
:102930000D51E8240101C7130E010E510101C71307
:10294000C86BC96BCA6BCB6BCC6BCD6BC60EE66E1E
:10295000010EE66E7E0EE66E010EE66EF1EC0EF0F6
:10296000E552E552E552E552E76E060EE7CFDBFF92
:10297000DB50146E070EE15C02E2E16AE552E16EA3
:102980001450E552E7CFD9FF1200D9CFE6FFE1CFCF
:10299000D9FF0101006BFE0EDB50016F026B000ED0
:1029A0000127010E0223036B046B02AF02D00369FF
:1029B0000469050E056FFE0EDB50066F076B000EF7
:1029C0000627010E0723086B096B07AF02D00869C1
:1029D0000969126FFE0EDB50136F146B000E132784
:1029E000020E1423156B166B14AF02D0156916690D
:1029F000080E176F186B196B1A6B1B6B020E246F86
:102A0000FE0EDB50256F266B010E2527020E2623B6
:102A1000276B286B26AF02D027692869080E296F1B
:102A20002A6B2B6B2C6B2D6B030E366FFE0EDB505F
:102A3000376F386B020E37273823396B3A6B38AF54
:102A400002D039693A69080E3B6F3C6B3D6B3E6BB7
:102A50003F6B040E486FFE0EDB50496F4A6B030E4E
:102A60004927020E4A234B6B4C6B4AAF02D04B698D
:102A70004C69080E4D6F4E6B4F6B506B516B050ED2
:102A80005A6FFE0EDB505B6F5C6B040E5B27020E11
:102A90005C235D6B5E6B5CAF02D05D695E69080EA6
:102AA0005F6F606B616B626B636B060E6C6FFE0E2B
:102AB000DB506D6F6E6B050E6D27020E6E236F6B14
:102AC000706B6EAF02D06F697069080E716F726BB8
:102AD000736B746B756B070E7E6FFE0EDB507F6F32
:102AE000806B060E7F27020E8023816B826B80AF86
:102AF00002D081698269080E836F846B856B866B57
:102B0000876B906FFE0EDB50916F926B070E9127D3
:102B1000020E9223936B946B92AF02D093699469E7
:102B2000080E956F966B976B986B996BA26FFE0E64
:102B3000DB50A36FA46B0A0EA327020EA423A56B80
:102B4000A66BA4AF02D0A569A669080EA76FA86BF3
:102B5000A96BAA6BAB6B010EE552E7CFD9FF120050
:102B6000800EE66EC2DAE5520E01010E436FF80EDA
:102B7000446F440E456F200E706E729E728C606AB8
:102B80000F01306B0E01806B906BA06BB06BC06B54
:102B9000D06BF80E7D6F880EE06F220EE16FE46F50
:102BA000080EE56F140EE86F050EE96F070E466F0D
:102BB000476B716B110E726F736F746B756B766B05
:102BC000776B786B500E796F050E7A6F7B6B7B6B32
:102BD000F869F969F997FC6BFD6BFD97E66A85DA90
:102BE000E5521200D9CFE6FFE1CFD9FF1A0EE12658
:102BF000D950060FE96EDACFEAFF200EEE6E0F0E07
:102C0000ED6ED950080FE96EDACFEAFF100EEE6EC6
:102C10000F0EED6ED9500A0FE96EDACFEAFF000E03
:102C2000EE6E0F0EED6ED9500C0FE96EDACFEAFFA3
:102C3000800EEE6E0E0EED6ED9500E0FE96EDACFED
:102C4000EAFF900EEE6E0E0EED6ED950100FE96E8B
:102C5000DACFEAFFA00EEE6E0E0EED6ED950120F17
:102C6000E96EDACFEAFFB00EEE6E0E0EED6ED950C1
:102C7000140FE96EDACFEAFFC00EEE6E0E0EED6EA7
:102C8000D950160FE96EDACFEAFFD00EEE6E0E0EB7
:102C9000ED6E0E017D417F0BE76E190EE7CFDBFF76
:102CA000DF6ADF50146E156A080E145C000E1558AA
:102CB00001E3DED0D950060F146EDF50020D145020
:102CC000F324E96EDA50F420EA6E020EEECFDBFF59
:102CD000030EEDCFDBFF020EDBCF08F0030EDBCFE0
:102CE00009F0040E08C0DBFF050E09C0DBFFDF5052
:102CF000020810E2190EDBCFF3FFF390F342F3CF9B
:102D0000DBFFD950190FE96EDACFEAFFEF50010B64
:102D100001E1ACD0020EDBCFE9FF030EDBCFEAFF0F
:102D2000EF50080B01E0A2D0FC0E146E020EDBCFB8
:102D3000E9FF030EDBCFEAFF1450EF16F70EDB506E
:102D4000030B146E020EDBCFE9FF030EDBCFEAFFAD
:102D50001450EF12F70EDBAC04D0F80EDB50400934
:102D600002D0F80EDB50E76E180EE7CFDBFF050E42
:102D7000E76E020EDBCFE9FF030EDBCFEAFFE75081
:102D8000E926000EEA22180EDBCFEFFFF70EDBAAD2
:102D900006D0010EF36E180EF3CFDBFF02D0180E33
:102DA000DB6ADBCFE6FFD950FB0FE96EFF0EDA20BE
:102DB000EA6EEECFE6FFEECFE6FFEECFE6FFEFCF17
:102DC000E6FF010EE76E020EDBCF14F0030EDBCF41
:102DD00015F0E7501426000E152214C0E6FF15C0AA
:102DE000E6FF97D9166E070EE15E1650D950020F16
:102DF000E96EDACFEAFF060EEE26000EED22010E96
:102E0000DB6AF80EDB50F36E010EDBCFF4FFF350FC
:102E1000F45C1AE2F90EDBCFE9FFDB2AFA0EDBCF16
:102E2000EAFF01E3DB2AEF50E66E020EDBCFE9FF9B
:102E3000DB2A030EDBCFEAFF01E3DB2AE552E75092
:102E4000EF6E010EDB2ADDD7040EDBCFE9FF050EA6
:102E5000DBCFEAFFEF50040B07E1040EDBCFE9FF05
:102E6000050EDBCFEAFFEF86010E03D0DF2A19D76C
:102E7000000E146E1A0EE15C02E2E16AE552E16EA8
:102E80001450E552E7CFD9FF1200D9CFE6FFE1CFCA
:102E9000D9FF060EE1260E010F6B60AE04D0600E66
:102EA000DE6E0F0E43D00F0130AF04D0300EDE6E59
:102EB0000F0E3CD00E017D51040B07E18051800BB9
:102EC00004E0800EDE6E0E0E31D07D51080B07E15E
:102ED0009051800B04E0900EDE6E0E0E27D07D51D7
:102EE000100B07E1A051800B04E0A00EDE6E0E0E69
:102EF0001DD07D51200B07E1B051800B04E0B00ED6
:102F0000DE6E0E0E13D07D51400B07E1C051800BD9
:102F100004E0C00EDE6E0E0E09D07D51800B13E171
:102F2000D051800B10E0D00EDE6E0E0EDD6EDECFC7
:102F3000E9FFDDCFEAFFEF501F0B0E010F6F779215
:102F400071AC0BD002D0000EC4D0F70EDBCFE9FF7E
:102F5000F80EDBCFEAFFEF86719CD9CFE9FFDACF1D
:102F6000EAFF020EEECFDBFF030EEDCFDBFFF70E25
:102F7000DBCFE9FFF80EDBCFEAFFEF6ADECFE9FF38
:102F8000DDCFEAFF050EE926000EEA22050EEFCF9F
:102F9000DBFFDB500F0BE66EF90EDBCFE9FFFA0E1D
:102FA000DBCFEAFFE552E750EF6ED950050FE96E2F
:102FB000DACFEAFFEF50400B07E0F70EDBCFE9FF77
:102FC000F80EDBCFEAFFEF8CDECFE9FFDDCFEAFFC3
:102FD000020EE926000EEA22050EEFCFDBFFD950E4
:102FE000050FE96EDACFEAFFEF50080B0DE0F70EA0
:102FF000DBCFE9FFF80EDBCFEAFFEF8A010EF36EBD
:10300000050EF3CFDBFF02D0050EDB6ADBCFE6FF58
:10301000FD0EDBCFE6FFFE0EDBCFE6FFDECF14F0CA
:10302000DDCF15F0010E1426000E152214C0E6FFA8
:1030300015C0E6FF46D9166E050EE15E1650060E67
:10304000DE26000EDD22F90EDBCFE9FFFA0EDBCF24
:10305000EAFF050EEFCFDBFF040EDB6ADBCF14F0D7
:10306000156A14BE1568050EDB50000115AE02D0BE
:10307000D89003D0145C000E155819E2DFCFE9FF99
:10308000DF2A010EDBCFEAFF01E3DB2AEF50E66E19
:10309000FB0EDBCFE9FFDB2AFC0EDBCFEAFF01E30F
:1030A000DB2AE552E750EF6E040EDB2AD7D777AE66
:1030B00008D0F70EDBCFE9FFF80EDBCFEAFFEF8891
:1030C000779E020EDBCFE9FF030EDBCFEAFFEF9E18
:1030D000010E146E060EE15C02E2E16AE552E16E59
:1030E0001450E552E7CFD9FF1200D9CFE6FFE1CF68
:1030F000D9FF1F0E6F16FE0EDB506F12E00E6F141D
:10310000146EFE0EDB50145CF9E1E552E7CFD9FFF7
:103110001200D9CFE6FFE1CFD9FF020EE126D95048
:10312000F90F146EFF0EDA2014C0DEFFDD6EF80E0C
:10313000DB50146E156AE850151031E1DECFE9FF5F
:10314000DDCFEAFFEF50E840E840E8401F0BE66EB5
:10315000FD0EDBCFE9FFFE0EDBCFEAFFE552E750C5
:10316000EF6EDECFE9FFDDCFEAFFEE52EF50200D2C
:10317000F3CF14F0FD0EDBCFE9FFFE0EDBCFEAFF4D
:10318000F350EF12FD0EDB2AFE0E01E3DB2ADECF49
:10319000E9FFDDCFEAFFEF50200DF3507ED0DECF08
:1031A000E9FFDDCFEAFF020EE926000EEA22EF502A
:1031B000E00BE838E840E66EFD0EDBCFE9FFFE0EDF
:1031C000DBCFEAFFE552E750EF6EDECFE9FFDDCF60
:1031D000EAFF030EE926000EEA22EF50080DF3CFB6
:1031E00014F0FD0EDBCFE9FFFE0EDBCFEAFFF3505C
:1031F000EF12FD0EDB2AFE0E01E3DB2ADECFE9FF34
:10320000DDCFEAFF020EE926000EEA22EF50080D9C
:10321000F350E00BE66EFD0EDBCFE9FFFE0EDBCFD9
:10322000EAFFE552E750EF6EFD0EDBCFE9FFFE0E41
:10323000DBCFEAFFEF86DECFE9FFDDCFEAFF020E4C
:10324000E926000EEA22EF50030B146EFD0EDBCFD1
:10325000E9FFFE0EDBCFEAFF1450EF12FD0EDB2A72
:10326000FE0E01E3DB2ADECFE9FFDDCFEAFFEE52FF
:10327000EF50E66EFD0EDBCFE9FFFE0EDBCFEAFF7F
:10328000E552E750EF6EFD0EDB2AFE0E01E3DB2A6E
:10329000DECFE9FFDDCFEAFFEF50E66EFD0EDBCFBC
:1032A000E9FFFE0EDBCFEAFFE552E750EF6E020EBC
:1032B000E15C02E2E16AE552E16EE552E7CFD9FF57
:1032C0001200D9CFE6FFE1CFD9FF020EE126FB0EB7
:1032D000DBCFDEFFDBCFDDFFFA0EDB50156AE850F7
:1032E00015104CE1FD0EDBCFE9FFFE0EDBCFEAFF50
:1032F000EF50080DF350E66EDECFE9FFDDCFEAFFB9
:10330000E552E750EF6EFD0EDBCFE9FFFE0EDBCF9F
:10331000EAFFEF50E00BE838E840E66EDECFE9FF69
:10332000DDCFEAFFEE52E552E750EF6EFD0EDB2AED
:10333000FE0E01E3DB2AFD0EDBCFE9FFFE0EDBCF45
:10334000EAFFEF50E00BE838E840DECFE9FFDDCFE1
:10335000EAFFE850EF12DECFE9FFDDCFEAFF020E11
:10336000E926000EEA22EF6ADECFE9FFDDCFEAFFB1
:10337000030EE926000EEA22EF6A84D0FD0EDBCFB1
:10338000E9FFFE0EDBCFEAFFEF50200DF350E66EB3
:10339000DECFE9FFDDCFEAFF020EE926000EEA22CA
:1033A000E552E750EF6EFD0EDBCFE9FFFE0EDBCFFF
:1033B000EAFFEF50E840E840E8401F0BE66EDECF42
:1033C000E9FFDDCFEAFF030EE926000EEA22E5520F
:1033D000E750EF6EFD0EDB2AFE0E01E3DB2AFD0E49
:1033E000DBCFE9FFFE0EDBCFEAFFEF50030B146EDD
:1033F000DECFE9FFDDCFEAFF020EE926000EEA226A
:103400001450EF12FD0EDBCFE9FFFE0EDBCFEAFF1B
:10341000EF50E00BE840E840E8401F0B146EDECFB1
:10342000E9FFDDCFEAFF020EE926000EEA22145082
:10343000EF12FD0EDB2AFE0E01E3DB2AFD0EDBCFD1
:10344000E9FFFE0EDBCFEAFFEF50E66EDECFE9FFCD
:10345000DDCFEAFFEE52E552E750EF6EFD0EDB2ABC
:10346000FE0E01E3DB2AFD0EDBCFE9FFFE0EDBCF14
:10347000EAFFEF50E66EDECFE9FFDDCFEAFFE5526F
:10348000E750EF6E020EE15C02E2E16AE552E16EA6
:08349000E552E7CFD9FF12005D
:08349800DACFE4FFE2CFDAFF16
:1034A000E9CFE4FFEACFE4FFF6CFE4FFF7CFE4FF94
:1034B000F5CFE4FFF3CFE4FFF4CFE4FFFACFE4FF6E
:1034C00000EE00F0140EE80403E3EECFE4FFFBD7B8
:1034D00000EE14F00E0EE80403E3EECFE4FFFBD79A
:1034E000E6529D50010B01E1B8D09E50010B01E165
:1034F000B4D0B20ECF6ECE6A9E90E0C122F0E1C190
:1035000023F0E2C124F0E3C125F0030E0B6E0C6A38
:103510000D6A0E6AE0C106F0E1C107F0E2C108F0F1
:10352000E3C109F03FEC1FF0025003100410051036
:1035300002E10101D381E0C122F0E1C123F0E2C147
:1035400024F0E3C125F00A0E0B6E0C6A0D6A0E6AB8
:10355000E0C106F0E1C107F0E2C108F0E3C109F003
:103560003FEC1FF0025003100410051009E10101A7
:10357000D3838D72040ED75D03E1DE2B000EDF23B3
:10358000050E0101E01907E1E15105E1E25103E116
:10359000E35101E1D385080EE01907E1E15105E1AE
:1035A000E25103E1E35101E1D3850B0EE01907E19C
:1035B000E15105E1E25103E1E35101E1D3850E0E52
:1035C000E01907E1E15105E1E25103E1E35101E1D5
:1035D000D385110EE01907E1E15105E1E25103E164
:1035E000E35101E1D385140EE01907E1E15105E152
:1035F000E25103E1E35101E1D385E0C122F0E1C1F1
:1036000023F0E2C124F0E3C125F0640E0B6E0C6AD6
:103610000D6A0E6AE0C106F0E1C107F0E2C108F0F0
:10362000E3C109F03FEC1FF002C022F003C023F019
:1036300004C024F005C025F002500310041005104A
:1036400006E10101D387E06BE16BE26BE36B010103
:10365000E02B000EE123E223E3237750020B1CE072
:103660007650020B19E00101100EDC6F779292EC9C
:103670000FF070EC10F03FEC14F03BEC11F0010196
:10368000DE6BDF6BD52BD62B080ED55D01E3D56B3A
:10369000060ED65D01E3D66BE55200EE21F00E0E6C
:1036A000E80403E3E5CFEDFFFBD700EE13F0140EC3
:1036B000E80403E3E5CFEDFFFBD7E5CFFAFFE5CF65
:1036C000F4FFE5CFF3FFE5CFF5FFE5CFF7FFE5CF5B
:1036D000F6FFE5CFEAFFE5CFE9FFE5CFDAFF11001E
:1036E000D9CFE6FFE1CFD9FFE652D050DF6E000E12
:1036F000DB94DB9CDB9EDF501B0A0EE0300A0BE004
:10370000110A08E0020A05E00B0A01E006D00400F5
:1037100005D004D003D002D001D000D03F0ED0128B
:1037200022EC00F0FE0EDBCFD7F1E552E552E7CFF9
:10373000D9FF1200D9CFE6FFE1CFD9FF070EE1266E
:10374000DE6ADD6A020EDB6A030EDB6A040EDB6AE8
:10375000050EDB6A060EDB6A0101D751100A01E192
:1037600063D1180A01E156D10C0A01E187D0060A9B
:1037700001E17AD0220A10E0210A01E085D1FDECB6
:1037800010F0040E0101D75D06E1789276827792FF
:103790000E010F0E7E6F79D1E66A50EC1DF0E552F6
:1037A000E76E020EE7CFDBFF0101020ED76F020EBC
:1037B000DB50AA0803E00101100ED76FD7C1E6FF66
:1037C0008FDFE5525DEC0DF0F3CF14F0F4CF15F080
:1037D000166A176A15AE02D016681768030E14C071
:1037E000DBFF040E15C0DBFF050E16C0DBFF060E67
:1037F00017C0DBFFD950030FE96EDACFEAFFD8908C
:10380000030EEB50000A08E6440EEE5C090EEE587B
:10381000000EEE58000EEE5802E3000E01D0010E2D
:10382000146E030EDBCF07F0040EDBCF08F0050E9D
:10383000DBCF09F0060EDBCF0AF00A34000E0A18BF
:1038400009E6D8803E0E07540A0E0854000E0954AB
:10385000000E0A5402E3000E01D0010E141003E022
:103860000E01010E086F11D1ECEC03F0F3CFDEFF77
:10387000F4CFDDFF0101010ED76F07D10101D35154
:10388000010B0BE00101D3910101D351100B03E0B7
:103890005AEC0DF002D00101D3890101D351020B82
:1038A00002E00101D3930101D351040B0BE00101AC
:1038B000D3950101D351400B03E05AEC0DF002D037
:1038C0000101D38D0101D351080B5EE00101D397B3
:1038D000040E0101DB5D03E30101080ED76F0E0149
:1038E000086B5DEC0DF0F3CF14F0F4CF15F0166A11
:1038F000176A15AE02D016681768030E14C0DBFFF6
:10390000040E15C0DBFF050E16C0DBFF060E17C048
:10391000DBFFD950030FE96EDACFEAFFD890030E30
:10392000EB50000A08E6440EEE5C090EEE58000E5D
:10393000EE58000EEE5802E3000E01D0010E146E98
:10394000030EDBCF07F0040EDBCF08F0050EDBCF54
:1039500009F0060EDBCF0AF00A34000E0A1809E659
:10396000D8803E0E07540A0E0854000E0954000E6B
:103970000A5402E3000E01D0010E141003E00E0100
:10398000010E086F0101DB6B0101D351A00B39E17E
:1039900001010A0ED880DE55000EDF5507E2010155
:1039A000CF6BD06BD16BD26B3BEC02F0100E0101F0
:1039B000DC5D27E10101200EDC6FCFC114F0D0C126
:1039C00015F0D1C116F0D2C117F0141E151E161E27
:1039D000171E14C0E6FF15C0E6FF16C0E6FF17C0AD
:1039E000E6FFCFC1E6FFD0C1E6FFD1C1E6FFD2C1FD
:1039F000E6FF010EE66EE3EC05F0186E090EE15EDF
:103A00001850D30EE66E010EE66ECBEC00F0E552D8
:103A1000E5523BD0FC0E8D148D6E0101010EDD6F61
:103A20000101040ED76F31D00101DD052AE1030E3B
:103A30008D12F29EF29C76920101040EDD6FE66A11
:103A4000E6680D0EE66EE66AE66AF80EE66E0E0EA3
:103A5000E66E89EC18F0146E070EE15E14500E014C
:103A60004681E66AE66A010EE66EE66AE66AE00EFE
:103A7000E66E0E0EE66E89EC18F0146E070EE15E2F
:103A80001450D6EC11F001D000D00400070EE15C18
:103A900002E2E16AE552E16EE552E7CFD9FF12009A
:103AA000D9CFE6FFE1CFD9FF020EE126010EDB6A96
:103AB000DE52120EDD6EFE0EDB50DF6EDF6A010E8F
:103AC000DB50DF5C10E2DF50746E7F9E7F9C7F8056
:103AD0000000DF50EA6AE40FE96E010EEA2273CFBC
:103AE000EFFFDF2AECD70101E45100D0146E020E83
:103AF000E15C02E2E16AE552E16E1450E552E7CF83
:103B0000D9FF1200D9CFE6FFE1CFD9FF090EE12698
:103B1000010EDB6A020EDB6A030EDB6A040EDB6A4F
:103B2000050EDB6A060EDB6A070EDB6A080EDB6A2F
:103B3000FE0EDB5027E1010EDB6A080EF36E010E6C
:103B4000DBCFF4FFF350F45C01E32ED1010EDB5028
:103B5000E76EFC0EDBCFE9FFFD0EDBCFEAFFE7509F
:103B6000E926000EEA22EF50E66E010EDB28EA6A33
:103B7000E40FE96E010EEA22E552E750EF6E010E06
:103B8000DB2ADBD7FE0EDB50080801E00DD1010E69
:103B9000DB6A040EF36E010EDBCFF4FFF350F45C2E
:103BA0001DE2010EDB50E76EFC0EDBCFE9FFFD0EE0
:103BB000DBCFEAFFE750E926000EEA22EF50E66E7F
:103BC000010EDB50090FEA6AE40FE96E010EEA22EA
:103BD000E552E750EF6E010EDB2ADBD70101AA0E9A
:103BE000E46FF16B300EE55D1A6E1B6A300EE65D18
:103BF0001C6E1D6A0A0E086E096A1CC00DF01DC0FD
:103C00000EF073EC1FF01A500624186E1B5007209C
:103C1000196E300E0101E75D1E6E1F6A640E086E9C
:103C2000096A1EC00DF01FC00EF073EC1FF0185093
:103C30000624166E19500720176E300E0101E85D3C
:103C4000206E216AE80E086E030E096E20C00DF08A
:103C500021C00EF073EC1FF016500624146E17509E
:103C60000720156EFF0E1416000E1516030E14C055
:103C7000DBFF040E15C0DBFF300E0101E55D1A6E9F
:103C80001B6A300EE65D1C6E1D6A0A0E086E096A1C
:103C90001CC00DF01DC00EF073EC1FF01A5006246E
:103CA000186E1B500720196E300E0101E75D1E6E65
:103CB0001F6A640E086E096A1EC00DF01FC00EF068
:103CC00073EC1FF018500624166E19500720176E5B
:103CD000300E0101E85D206E216AE80E086E030EC9
:103CE000096E20C00DF021C00EF073EC1FF01650CD
:103CF000062417500720146E156A050E14C0DBFF4A
:103D0000060E15C0DBFF300E0101EB5D0A0D300E13
:103D1000EA5DF324E76E070EE7CFDBFF300EEE5DC2
:103D20000A0D300EED5DF324E76E080EE7CFDBFFE2
:103D3000030EDBCFF2F1050EDBCFF3F1070EDBCF85
:103D4000F4F1080EDBCFF5F1120EF36E020EF3CF95
:103D5000DBFF010EDB6A020EDB50F36E010EDBCFE0
:103D6000F4FFF350F45C20E2010EDB50746E010EA0
:103D7000DB50EA6AE40FE96E010EEA22EF50736E3F
:103D80007F9E7F9C7F84F250DF6EF26A550E7E6EBE
:103D9000AA0E7E6E7F82DF50F26E7F94B7ACFED7A4
:103DA000B79C010EDB2AD7D7090EE15C02E2E16A7B
:103DB000E552E16EE552E7CFD9FF1200D9CFE6FF19
:103DC000E1CFD9FFE652FE0EDB50746EFD0EDB50E4
:103DD000736E7F9E7F9C7F84F250DF6EF26A550E79
:103DE0007E6EAA0E7E6E7F82DF50F26E7F94B7AC3D
:0E3DF000FED7B79CE552E552E7CFD9FF12008F
:023DFE00006A59
:103E00000EAE05EF1FF00E6C001E09AE0AEF1FF09C
:103E1000096C001E48EC21F009BE14EF1FF000AE43
:103E2000000C096C056C000C00BE11EF1FF001883E
:103E3000FF0C006A0EAE22EF1FF00D6C0E1EE86A3A
:103E40000E22001E09AE2AEF1FF0086C091EE86A58
:103E50000922001EF6EC20F009BE3AEF1FF000AE7A
:103E6000000C086C091EE86A0922046C051EE86A49
:103E70000522000C00BE31EF1FF00188FF0C006A24
:103E8000E86A0EAE4CEF1FF00B6C0C1E0D1E0E1EE2
:103E90000C220D220E22001E09AE57EF1FF0066CF9
:103EA000071E081E091E072208220922001EBBEC5D
:103EB00020F009BE6EEF1FF000AE000C066C071E6E
:103EC000081E091EE86A072208220922026C031E46
:103ED000041E051E032204220522000C00BE5EEF14
:103EE0001FF00188FF0C08C012F008500D02F4CF3B
:103EF00007F0F3CF06F009500E02F4CF09F0F3CF2C
:103F000008F00D02F3500726F4500822E86A09224F
:103F100012500E02F3500726F4500822E86A0922D4
:023F2000000C93
:0E3F22009F119711901188117F1176116D116A
:103F3000641159114F11441138112C111F11121114
:103F40000411F610E710D710C710B610A510921084
:103F50007F106C10571042102C101610FF0FE70F37
:103F6000CE0FB40F990F7D0F610F440F260F070F6F
:103F7000E80EC80EA70E850E620E3F0E1B0EF60D44
:103F8000D10DAB0D850D5E0D360D0D0DE40CBB0C8A
:103F9000910C670C3C0C120CE60BBA0B8F0B620BEE
:103FA000360B090BDD0AB00A830A570A2B0AFE09F1
:103FB000D109A50979094D092109F508CA089E0802
:103FC000740849081F08F507CC07A3077A075307A9
:103FD0002B070407DE06B80693066E064A06260679
:103FE0000306E105BF059E057D055D053E051F0530
:103FF0000005E204C504A9048D04710456043C04C0
:1040000023040A04F103D903C203AB0394037F031F
:104010006903550340032C0319030603F402E2026B
:10402000D002BF02AE029E028E027E026F026002CA
:0E40300052024402360229021B020F02030252
:02403E001E0E54
:10404000F66E000EF76E000EF86E01010900F550D5
:10405000FB6F0900F550FC6F03E1FB6701D03DD019
:104060000900F550F66F0900F550F76F0900F5509B
:10407000F86F09000900F550E96E0900F550EA6E85
:10408000090009000900F550F96F0900F550FA6FB1
:1040900009000900F6CFFDF1F7CFFEF1F8CFFFF1EF
:1040A000F6C1F6FFF7C1F7FFF8C1F8FF0101F953B8
:1040B00002E1FA5307E00900F550EE6EF907F8E265
:1040C000FA07F9D7FDC1F6FFFEC1F7FFFFC1F8FF00
:0C40D0000101FB07000EFC5BBFD71200D3
:0440DC00D9CFE6FF53
:1040E000E1CFD9FF020EE126CD0EDF6E010EDB6AB5
:1040F000FD0EDBCF14F0FE0EDBCF15F0D89015507F
:1041000004E6040E145C020E155803E25B0EDF6E2B
:1041100025D0010EF76ADB34FE0BF736F66E220E61
:10412000F6263F0EF7220900F5CF14F00800F5CF70
:1041300015F0FD0EDBCF16F0FE0EDBCF17F015509D
:104140001718E8AE02D0173404D01650145C17507C
:10415000155804E3010EDB2ADF2ADBD7DF50146E8B
:10416000020EE15C02E2E16AE552E16E1450E552B2
:06417000E7CFD9FF1200A9
:0A417600056A046A036A026A200E5B
:10418000E76ED8900636073608360936023603360B
:10419000043605360B50025C0C5003580D50045881
:1041A0000E50055809E30B50025E0C50035A0D5097
:0E41B000045A0E50055A062AE72EE4D71200D4
:0241BE00FF0EF2
:1041C000E350276EEF0E01D0F30EE76EE72EE6EF19
:1041D00020F00C0E266EE76AE72EECEF20F0262E7C
:0C41E000EBEF20F0272EE4EF20F012009F
:0441EC00056A046AF2
:1041F000100EE76ED89008360936043605360D5095
:10420000045C0E50055805E30D50045E0E50055A2F
:08421000082AE72EF0D7120086
:08421800FF0EE350276E480E73
:1042200001D04C0EE76EE72EFED7E76AE72EFED7E9
:08423000272EF7D70000120051
:08423800410EF36E00EE00F0F0
:104240000E0E01D81200EA6002D0EE6AFCD7F350DD
:08425000E9601200EE6AFCD7E0
:084258001DEE00F02DEE00F058
:10426000F86A019C1FEC20F003EC00F09AEC1BF0C4
:04427000FBD7120066
:0C427400FF0EE350276E1B0E00D001D09F
:10428000200EE76EE72EFED7272EFAD700D01200B9
:10429000056A080EE76ED890093605360E50055CA3
:0C42A00002E3056E092AE72EF7D7120092
:0442AC00000000000E
:1042B00000000000200000000020010000000000BD
:0142C00000FD
:020000040030CA
:0100000015EA
:0100010013EB
:0100030020DC
:00000001FF
